:100000000C9439000C9456000C9456000C94560035
:100010000C9456000C9456000C9456000C94560008
:100020000C9456000C9456000C9456000C945600F8
:100030000C9456000C9456000C9456000C945600E8
:100040000C9456000C9456000C9456000C945600D8
:100050000C94560005A84CCDB2D44EB93836A9023E
:100060000C50B9918688083CA6AAAA2ABE000000B6
:10007000803F11241FBECFE5D4E0DEBFCDBF10E02E
:10008000A0E6B0E0E4E5F9E102C005900D92A03EE3
:10009000B107D9F711E0A0EEB0E001C01D92A43F76
:1000A000B107E1F70E9450030C94A80C0C940000D7
:1000B000CF93DF9300D0CDB7DEB7AD98811102C0EA
:1000C000AC9801C0AC9AAD9A25B3862F992787FDCD
:1000D0009095807F99279595879595958795959586
:1000E000879595958795922F907F892B85BBAD98A5
:1000F000AD9A85B36F70807F682B65BBAD98CA01E0
:10010000880F991F480F591F440F551F440F551F43
:10011000440F551F5A83498389819A81892B49F05D
:1001200089819A8101979A83898389819A81892B10
:10013000B9F70F900F90DF91CF910895CF93DF9390
:10014000FC016081662351F0EC01219642E050E011
:1001500081E00E94580069916111F8CFDF91CF9141
:10016000089544E050E068E280E00E94580044E0D6
:1001700050E068E280E00E94580044E050E068E20D
:1001800080E00E94580048EC50E062E080E00E946D
:10019000580044E050E06CE080E00E94580040E8E5
:1001A00050E061E080E00E94580044E050E066E0EA
:1001B00080E00E94580008958A3040F4682F605D06
:1001C00042E050E081E00E9458000895682F695C89
:1001D00042E050E081E00E9458000895CF93C82F7C
:1001E00082958F700E94DC008C2F8F700E94DC0043
:1001F000CF910895CF93C82F892F0E94EE008C2FA6
:100200000E94EE00CF910895CF93DF93C82FD9E2DB
:100210008D9FD12D1124D295DF706D2F605D42E04E
:1002200050E081E00E94580084E6D89FC019112454
:10023000DDECCD9FD12D1124D695D695D6956D2F79
:10024000605D42E050E081E00E945800DD0F8D2F9C
:10025000880F880FD80FCD1B6C2F605D42E050E0F7
:1002600081E00E945800DF91CF9108950F931F9372
:10027000CF93DF938C019C01329522952F70232719
:100280003F702327A7E4B3E00E94790CEC01D695D8
:10029000C795D695C795D695C7956C2F605D42E0FA
:1002A00050E081E00E94580020E137E2C29FC00187
:1002B000C39F900DD29F900D1124081B190B98011C
:1002C000369527953695279536952795A5ECB0E276
:1002D0000E94790CEC01D295C295CF70CD27DF70CA
:1002E000CD276C2F605D42E050E081E00E94580015
:1002F00028EE33E0C29FC001C39F900DD29F900DA6
:100300001124081B190B98013695279536952795CA
:10031000ABE7B4E10E94790CEC01D695C7956C2F40
:10032000605D42E050E081E00E94580024E62C9F8E
:10033000C0012D9F900D1124081B190B9801ADECE5
:10034000BCEC0E94790CEC01D695C795D695C79563
:10035000D695C7956C2F605D42E050E081E00E9429
:100360005800CE01880F991FCC0FDD1FCC0FDD1F69
:10037000CC0FDD1FC80FD91F0C1B1D0B602F605D3C
:1003800042E050E081E00E945800DF91CF911F9140
:100390000F910895EF92FF920F931F93CF93DF93E6
:1003A00000E0C0E0D0E0F12C16C0612F6E2944E0DF
:1003B00050E08F2D0E9458004AE050E0602F81E00D
:1003C0000E9458001F5F183081F706950061219642
:1003D000C530D10569F09E01220F331F220F331F54
:1003E000220F331F6894EE24E6F8E22A1F2DDDCF9A
:1003F000DF91CF911F910F91FF90EF9008959F9201
:10040000AF92BF92CF92DF92EF92FF920F931F9322
:10041000CF93DF93E12CF12CA12CB12C0F2EF7E020
:10042000CF2ED12CF02D22C06C2F692944E050E052
:1004300080E00E9458000C171D073CF04AE050E095
:1004400060E081E00E94580006C04AE050E06FEF93
:1004500081E00E9458002196C830D10529F78FEF1E
:10046000E81AF80A88E0E816F10481F0C701880F5D
:10047000991F880F991F880F991F6894992496F8DF
:10048000982AE50186010E191F09CECFDF91CF9181
:100490001F910F91FF90EF90DF90CF90BF90AF90A2
:1004A0009F900895DF92EF92FF920F931F93CF9347
:1004B000DF93D82EAB0181E08D1508F484C09B0139
:1004C000ADECBCEC0E94790CEC01D695C795D695A5
:1004D000C795C031D10508F04EC08E01CE01880FFE
:1004E000991F880F991F080F191FCA01801B910BB4
:1004F0008C01D0FAEE24E0F8F12C0024F694E79475
:100500000794F694E7940794FE2CE02C6894E7F89F
:10051000FF24FA946D2D6270660F660F660F6E29C8
:1005200044E050E080E00E945800209709F040C06D
:1005300042C042E050E06FEF81E00E945800F39427
:100540002F2D332727FD3095C217D30790F742E0B0
:1005500050E0602F81E00E945800CF2DCF5FC13165
:1005600094F542E050E060E281E00E945800CF5FE5
:10057000C131BCF328C0ED2DE170F0E00024F69508
:10058000E7950794F695E7950794FE2FE02DE06830
:10059000FF6F6D2D6270660F660F660F6E2B44E065
:1005A00050E080E00E94580000E010E0CFE0D0E092
:1005B000FF24F394BECF42E050E0602F81E00E9420
:1005C0005800C2E0CECFDF91CF911F910F91FF90E5
:1005D000EF90DF9008951F93CF93DF93C82F883259
:1005E00048F56830710518F4D62F10E209C0603163
:1005F000710520F4162F1770DFEF02C0DFEF1FEF39
:100600006C2F606844E050E080E00E94580042E0B7
:1006100050E0612F81E00E9458006C2F606C44E034
:1006200050E080E00E94580042E050E06D2F81E0F1
:100630000E945800DF91CF911F910895CF93DF93CF
:10064000EA01683250F5982F9270990F990F990F1F
:10065000692B282F217030E00024369527950794C8
:10066000369527950794322F202D20683F6F622BF7
:1006700044E050E080E00E945800C830D10538F4D2
:1006800042E050E06C2F81E00E94580006C042E03A
:1006900050E06FEF81E00E945800DF91CF91089504
:1006A000CF93DF93CDB7DEB7E6970FB6F894DEBFF2
:1006B0000FBECDBF1C821B828B819C8142977CF533
:1006C0000B811C816B817C816F5F7F4F882777FD59
:1006D0008095982F0E94640A2BED3FE049EC50E48E
:1006E0000E94010B20E030E040E05CE30E94010B3F
:1006F0000E942E0A00521F4F20E030E04EEF52E4DD
:100700000E94010B0E94310AD8016C938B819C815D
:1007100001969C838B838B819C8142978CF28FEF17
:1007200084BB81BB82BB88BB8CEF8BBB0E94B100BA
:100730000E94FF0182E18CBF8BE083BF8BE687B90B
:1007400085E086B980E680BF86B1806E86B944E0D8
:1007500050E062E880E00E9458008CE990E00E943E
:100760009E0044E050E066EC80E00E94580089EA78
:1007700090E00E949E0086B38F3FE9F386B38F3FDF
:10078000E9F7B1E0BCA7E6E0EBA7F9E0FBA327E0BF
:100790002B8F31E0388F41E04F8B1FA618AA19AA82
:1007A0001AAA81E090E09A83898389819A819C01C9
:1007B0002F5F3F4F3A832983813891050CF071C137
:1007C0001D821E821F82188619861A861B861C8629
:1007D000212C312C00E010E0F0E0E0E01D861E86C8
:1007E000C12CD12C76011F861B8A1C8A1D8A1E8A69
:1007F0000CC0242E352E062F172FF82DE92DAD868F
:10080000BE864F865B8A6C8A7D8A349BFECFA98127
:10081000BA8184B195B1AA0FBB1FAE50BF4F8D9363
:100820009C93349A88B7826088BFA981BA81AA0F45
:10083000BB1FAE50BF4F8D919C918115904861F0C8
:10084000A981BA81AA0FBB1FAE50BF4F8D919C9159
:10085000803C9F4731F403C02F892E8B02C03F8913
:100860003E8BA981BA81AA0FBB1FAE50BF4F8D919D
:100870009C911197082E892F000C881F990B000C52
:10088000881F991F8D939C9389819A81819734F554
:10089000A981BA8189819A81A980BA80AA0FBB1FD8
:1008A0009D012E503F4F880F991F8E509F4FDC01A6
:1008B0006D917C91A69EC001A79E900DB69E900D55
:1008C00011249595879595958795959587959595F7
:1008D000879595958795D9018D939C9389819A8168
:1008E0008136910554F1A981BA8189819A81298142
:1008F0003A81AA0FBB1FBD016E507F4F880F991F11
:100900008E509F4F41E850E0421B530BDC012D916C
:100910003C91429FC001439F900D529F900D112426
:1009200095958795959587959595879595958795AF
:1009300095958795DB018D939C93A9EEB0E08C9102
:10094000A82FBB27A7FDB0952F853B894C895D89D2
:100950000E94850C2B013C01689415F875946794EE
:10096000579447941694D1F74C185D086E087F0889
:10097000A981BA81AA0FBB1FAE50BF4F8D919C9128
:10098000AA2797FDA095BA2F480E591E6A1E7B1EF6
:10099000A8EEB0E08C91A82FBB27A7FDB0952F2F14
:1009A0003E2F4D855E850E94850C4B015C0168944D
:1009B00015F8B594A794979487941694D1F7298540
:1009C0003A854B855C85821A930AA40AB50AA981E7
:1009D000BA81AA0FBB1FAE50BF4F8D919C91AA2721
:1009E00097FDA095BA2F880E991EAA1EBB1EAAEECF
:1009F000B0E08C91A82FBB27A7FDB095222D332DF9
:100A0000402F512F0E94850CAB01BC01689415F852
:100A100075956795579547951694D1F78D819E8169
:100A2000AF81B885481B590B6A0B7B0BA981BA8132
:100A3000AA0FBB1FAE50BF4F8D919C91AA2797FD67
:100A4000A095BA2F480F591F6A1F7B1F89819A8171
:100A50009C012F5F3F4F3A832983CF84DB88EC884A
:100A6000FD88F987EA87AD85AB87BE85BC872D8277
:100A70003E820F831887813891050CF4BACE4D83DE
:100A80005E836F8378872E89211123C029863E8A51
:100A9000098F1A8F3F2E2E2EFC2DED2D1E2D0F2D82
:100AA00016C019861E8A198E1A8E312C212C1D868D
:100AB0001E861D821E821F821886812C912C540155
:100AC000F0E0E0E010E000E0412C512C3201979A78
:100AD0000BC0979829863E8A098F1A8F3F2E2E2E9B
:100AE000FF85EB891C890D89288D21118BC2A301FB
:100AF0009201C301B2010E948D0C6B017C012F2F6A
:100B00003E2F412F502F6F2F7E2F812F902F0E942D
:100B10008D0CC60ED71EE81EF91EA30192016F2F81
:100B20007E2F812F902F0E948D0C9B01AC01E9EE4E
:100B3000F0E0A081BB27A7FDB0950E94850CDC01E9
:100B4000CB01689415F8B595A79597958795169458
:100B5000D1F7A7019601281B390B4A0B5B0B2F8796
:100B6000388B498B5A8B8C8D9D8DAE8DBF8D8115A9
:100B7000E0EE9E07E1E0AE07B10508F44CC0811538
:100B8000F0E29F07F3E0AF07B10508F048C02CA1E1
:100B90003DA14EA15FA182179307A407B507B8F442
:100BA0002F85388949895A8982179307A407B50781
:100BB00070F469017A018CA19DA1AEA1BFA1281793
:100BC00039074A075B07E0F56C017D0139C02C8DC0
:100BD0003D8D4E8D5F8D8CA19DA1AEA1BFA18217D1
:100BE0009307A407B50718F58F859889A989BA894D
:100BF00082179307A407B507F8F46C017D012CA1B7
:100C00003DA14EA15FA1281739074A075B07C0F431
:100C100069017A0115C0C12CD12C760111C00F2EAB
:100C2000C12CD12CF5E0EF2EF12CF02D09C0CC8C8D
:100C3000DD8CEE8CFF8C04C0CC8CDD8CEE8CFF8CBC
:100C4000A5019401C501B4010E948D0C2B013C014A
:100C5000232D322D4D855E85632D722D842F952F8A
:100C60000E948D0C460E571E681E791EA501940128
:100C7000632D722D8D859E850E948D0C9B01AC018C
:100C8000E8EEF0E0A081BB27A7FDB0950E94850C9F
:100C9000DC01CB01689415F8B595A79597958795D4
:100CA0001694D1F7481A590A6A0A7B0AF1E04F16DE
:100CB000F0E85F06F2E06F06710410F0929801C050
:100CC000929A2D813E814F815885CA01B9010E94B7
:100CD0008D0C4B015C0129853E89498D5A8D622F0F
:100CE000732F842F952F0E948D0C860E971EA81EA1
:100CF000B91E2D813E814F81588569857E89898DF8
:100D00009A8D0E948D0C9B01AC01EAEEF0E0A0816F
:100D1000BB27A7FDB0950E94850CDC01CB01689430
:100D200015F8B595A795979587951694D1F7881AD4
:100D3000990AAA0ABB0AF1E08F16F0E89F06F2E0D2
:100D4000AF06B10410F0909801C0909A21E0C2164D
:100D500020E8D20622E0E206F104A8F039A1311120
:100D600001C0919849A14F5F49A3CCA2DDA2EEA298
:100D7000FFA28F859889A989BA898C8F9D8FAE8FA4
:100D8000BF8F1AA247C299A19230A0F4AAA1A111C3
:100D900063C0919ACCA2DDA2EEA2FFA22F85388972
:100DA00049895A892C8F3D8F4E8F5F8F1AA618A2C2
:100DB00019A230C23AA131114FC04AA54F5F4AA7CC
:100DC00058A1550F58A38BA5882381F099A195317F
:100DD000C8F5ADA59A1708F49DA7BEA5E9A1BE1751
:100DE00008F4EEA7FBA5F150FBA72CC02CA52130E1
:100DF00049F54DA5242F30E05EA5852F90E0A9018F
:100E0000440F551F48175907C4F4820F931F959537
:100E100087958B8F99279C01220F331F220F331F39
:100E2000820F931F95958795959587958BA31EA601
:100E300084E18DA796E09BA705C01EA6A4E1ADA7FF
:100E4000B6E0BBA7E9A1FB8DFE1718F428A121602D
:100E500028A3919A19A203C03AA13F3F19F04AA1D1
:100E60004F5F4AA35AA1252F30E0ABA18A2F90E013
:100E700001962817390721F542E050E06FEF81E035
:100E80000E94580069A56270660F660F660FB8A5CC
:100E90006B2BE9A5E170EDAB1EAA8DA99EA90024DC
:100EA000969587950794969587950794982F802D0A
:100EB00080689F6F682B44E050E080E00E945800FB
:100EC000FAA12BA1F21388C13AA5313029F448A127
:100ED000411142C065E655C05AA5523039F488A187
:100EE000E82FF0E0E856FF4F60814BC09AA59330A1
:100EF00039F4A8A1EA2FF0E0E057FF4F608141C02C
:100F0000BAA5B43039F428A1E22FF0E0E058FF4F41
:100F1000608137C03AA5353039F448A1E42FF0E0BC
:100F2000E05AFF4F60812DC05AA55630B9F488A110
:100F30008531B1F08333B1F08833B1F08C30B1F04A
:100F40008131B1F08631B1F08D32B1F08A30B1F03B
:100F50008A31B1F460E415C064E713C060E211C0E7
:100F60006EE20FC06CE20DC06AE30BC06FE309C014
:100F70006DE207C068E205C069E203C06FE201C02C
:100F800060E242E050E081E00E94580088A58F5F57
:100F900098A59F3008F42DC1A9A58A2F90E001964D
:100FA0008170907889A79C012170332700243695A1
:100FB00027950794369527950794322F202D206882
:100FC0003F6F82709927880F991F880F991F880F8C
:100FD000991F622F682B44E050E080E00E94580087
:100FE000CCA2DDA2EEA2FFA22F85388949895A89B9
:100FF0002C8F3D8F4E8F5F8F3AA13BA31AA618A668
:1010000018A208C182E090E09C838B838B819C8135
:1010100042970CF0FFC07FA468A859A84AA841E0F5
:1010200050E05A83498389819A81813891050CF077
:1010300057C0C72CD62CE52CF42C072D162DF52DDA
:10104000E42D04C0082D192DFA2DEB2DAB81BC81A8
:10105000A052BF4FAC91AA0FBB0B202F312F4F2FA7
:101060005E2F0E94850C4B015C0199235CF40F2ECE
:10107000FFE78F2E912CA12CB12CF02D860E971E00
:10108000A81EB91E689416F8B594A79497948794EF
:101090001694D1F78C189D08AE08BF08A981BA81B3
:1010A000AA0FBB1FAE50BF4F8D919C91AA2797FDF1
:1010B000A095BA2F880E991EAA1EBB1E89819A81FF
:1010C00001969A83898389819A81C02ED12EEF2E31
:1010D000FE2E813891050CF4B5CF3F2E2E2E08C080
:1010E000072D162D352C242C872C962CA52CB42CB2
:1010F000EB81FC81A5019401C501B4010E948D0C16
:101100006B017C01202F312F432D522D602F712F29
:10111000832D922D0E948D0CC60ED71EE81EF91E3F
:10112000A5019401602F712F832D922D0E948D0CAB
:101130009B01AC01E052FF4FA081BB27A7FDB095FA
:101140000E94850CDC01CB01689415F8B595A79534
:10115000979587951694D1F7A7019601281B390B0F
:101160004A0B5B0BCA01B9010E94640AE62EF72EF6
:10117000082F192F44E050E067EC80E00E945800EF
:1011800042E050E06EE581E00E9458006E2D7F2D18
:10119000802F912F0E94680B0B811C8120E030E092
:1011A00040E250E40E94010B20E030E040E05CE3CC
:1011B0000E94010B0E94360A7727802F82500E94DE
:1011C000EB028B819C8101969C838B838B819C811C
:1011D00042970CF424CF1EC0CCA2DDA2EEA2FFA247
:1011E0008F859889A989BA898C8F9D8FAE8FBF8F83
:1011F00011C0CCA2DDA2EEA2FFA22F8538894989B9
:101200005A892C8F3D8F4E8F5F8F88A73AA13BA3C1
:101210001AA618A286B38F3F09F4C3CA16B31123C6
:101220000CF441C0488D413079F440E850E061E071
:1012300080E00E94580044E050E060E880E00E94B6
:10124000580019A618A606C180E291EAA7E0B0E00E
:10125000B79905C00197A109B109D1F704C0892B3D
:101260008A2B8B2B59F440E850E061E080E00E942B
:10127000580016FF1DC051E0588FA0C08B8D8230E2
:1012800010F081508B8FAB8D8A2F90E09C01220F44
:10129000331F220F331F820F931F959587959595C6
:1012A00087958BA3D7C016FD89C0B88DB13081F466
:1012B00040E850E061E080E00E94580044E050E0E7
:1012C00060E880E00E94580019A618A6188EBEC0DB
:1012D00080E291EAA7E0B0E0B69905C00197A109C4
:1012E000B109D1F705C0892B8A2B8B2B09F050C08F
:1012F000ECA5E11116C044E050E067EC80E00E94EC
:1013000058008FEA90E00E949E001EA6F4E1FDA71F
:1013100021E02CA736E03BA747E04BA356E05B8FCC
:101320000FC044E050E067EC80E00E94580089EB79
:1013300090E00E949E001CA686E08BA395E09B8F08
:10134000A8A5A73028F0B9A5B13011F419A618A6A0
:1013500069A56270660F660F660FE8A56E2BF9A58A
:10136000F170FBAB1CAA8BA99CA9002496958795CC
:101370000794969587950794982F802D80689F6F86
:10138000682B44E050E080E00E945800188E5EC058
:101390002B8D2F3010F42F5F2B8F3B8D832F90E000
:1013A0009C01220F331F220F331F820F931F95952D
:1013B0008795959587958BA3188E48C010FD46C0DC
:1013C00040E850E061E080E00E94580044E050E0D6
:1013D00060E880E00E94580083EC90E00E949E004C
:1013E00088EE93E00E94360186EC90E00E949E0019
:1013F0008B8D0E94040144E050E060EC80E00E948C
:1014000058008CEC90E00E949E008DA50E94040183
:101410008FEC90E00E949E008EA50E9404014CA5D6
:10142000413029F483ED90E00E949E0004C089EDD4
:1014300090E00E949E0086B38F3FE9F740E850E0BD
:1014400061E080E00E94580019A618A686B38F3F7D
:10145000E9F7A7C916FF3CCF188EB0CF71D0E3953E
:1014600096C004D06894B111C6C00895A9D088F080
:101470009F5790F0B92F9927B751A0F0D1F0660F80
:10148000771F881F991F1AF0BA95C9F712C0B1309B
:1014900081F0B0D0B1E00895ADC0672F782F8827D4
:1014A000B85F39F0B93FCCF3869577956795B395DA
:1014B000D9F73EF490958095709561957F4F8F4F49
:1014C0009F4F0895E89409C097FB3EF4909580954E
:1014D000709561957F4F8F4F9F4F9923A9F0F92FFA
:1014E00096E9BB279395F695879577956795B79578
:1014F000F111F8CFFAF4BB0F11F460FF1BC06F5F5E
:101500007F4F8F4F9F4F16C0882311F096E911C06F
:10151000772321F09EE8872F762F05C0662371F090
:1015200096E8862F70E060E02AF09A95660F771FA4
:10153000881FDAF7880F9695879597F908957AC1ED
:101540003FD0E8F3E894E0E0BB279F57F0F02AEDA6
:101550003FE049EC06C0EE0FBB0F661F771F881FE8
:1015600028F0B23A62077307840728F0B25A620B78
:10157000730B840BE3959A9572F7803830F49A9543
:10158000BB0F661F771F881FD2F7904847C1EF93A4
:10159000E0FF06C0A2EA2AED3FE049EC5FEBE3D0B2
:1015A00072D10F90039401FC9058E4E5F0E04CC137
:1015B00057FD9058440F551F59F05F3F71F0479504
:1015C000880F97FB991F61F09F3F79F087950895E9
:1015D000121613061406551FF2CF4695F1DF08C008
:1015E000161617061806991FF1CF86957105610525
:1015F00008940895E894BB2766277727CB0197F9CD
:1016000008950BD040C131D128F036D118F0952380
:1016100009F0FCC00FC11124EECFCADFA0F3959FE3
:10162000D1F3950F50E0551F629FF001729FBB27C9
:10163000F00DB11D639FAA27F00DB11DAA1F649F75
:101640006627B00DA11D661F829F2227B00DA11D28
:10165000621F739FB00DA11D621F839FA00D611DAE
:10166000221F749F3327A00D611D231F849F600DCF
:10167000211D822F762F6A2F11249F5750408AF008
:10168000E1F088234AF0EE0FFF1FBB1F661F771F94
:10169000881F91505040A9F79E3F510570F0B6C089
:1016A000AACF5F3FECF3983EDCF38695779567957C
:1016B000B795F795E7959F5FC1F7FE2B880F911DB2
:1016C0009695879597F9089511F40EF4B3C0A4C0C8
:1016D00077DFD0F39923D9F3CEF39F57550B87FFCC
:1016E000ACD00024A0E640EA90018058569597952A
:1016F00028F4805C660F771F881F20F026173707B5
:10170000480730F4621B730B840B202931294A2BC4
:10171000A69517940794202531254A2758F7660F78
:10172000771F881F20F026173707480730F4620B11
:10173000730B840B200D311D411DA09581F7B9015C
:10174000842F9158880F9695879508958ED030F004
:1017500093D020F031F49F3F11F41EF46BC00EF4CF
:10176000E095E7FB53C0E92F23DF80F3BA17620748
:1017700073078407950718F071F49EF53BCF0EF4BC
:10178000E0950B2EBA2FA02D0B01B90190010C0191
:10179000CA01A0011124FF27591B99F0593F50F4A9
:1017A000503E68F11A16F040A22F232F342F442701
:1017B000585FF3CF469537952795A795F0405395F9
:1017C000C9F77EF41F16BA0B620B730B840BBAF0C9
:1017D0009150A1F0FF0FBB1F661F771F881FC2F734
:1017E0000EC0BA0F621F731F841F48F48795779548
:1017F0006795B795F7959E3F08F0B3CF9395880FFF
:1018000008F09927EE0F97958795089597F99F67A8
:1018100080E870E060E008959F3F31F0915020F43F
:10182000879577956795B795880F911D96958795BC
:1018300097F908959FEF80EC089591505040660FFE
:10184000771F881FD2F708959F938F937F936F938D
:10185000FF93EF939B01AC01D4DEEF91FF9124D075
:101860002F913F914F915F91CCCE00240A94161690
:10187000170618060906089500240A94121613067E
:10188000140605060895092E0394000C11F488230C
:1018900052F0BB0F40F4BF2B11F460FF04C06F5F28
:1018A0007F4F8F4F9F4F0895DF93CF931F930F93D9
:1018B000FF92EF92DF927B018C01689405C0DA2ED3
:1018C000EF01ABDEFE01E894A5912591359145919C
:1018D0005591AEF3EF0147DFFE019701A801DA94BD
:1018E00079F7DF90EF90FF900F911F91CF91DF91EB
:1018F0000895A29FB001B39FC001A39F01D0B29FE2
:10190000700D811D1124911D0895B7FF0C949D0C3D
:101910000E949D0C821B930B0895DB018F939F9374
:101920000E949D0CBF91AF91A29F800D911DA39F1E
:10193000900DB29F900D112408950E94790CA59FDF
:10194000900DB49F900DA49F800D911D11240895BA
:04195000F894FFCF39
:1019540035345F335F5F5F325F5F2A5F5F5F5F31A4
:10196400362D2F5F5F5F5F5F375F5F5F385F3930B2
:10197400687666756C61706A627863797A716F688B
:1019840073757277646B676F69616E6D4D6F727397
:10199400654465636F64657200444B33504B007C4F
:1019A40053796E63206F6E20007C53796E63206FD1
:1019B400666600663D00206469743D006D3D00204C
:1019C4004D3D002053594F4E002053594F460000BF
:00000001FF
